:100000000EC026C025C024C023C022C021C020C0ED
:100010001FC01EC01DC01CC01BC01AC019C01124A7
:100020001FBECFEDCDBF20E0A4E6B0E001C01D9221
:10003000AD37B207E1F710E0A0E6B0E0E4ECF7E09E
:1000400002C005900D92A436B107D9F70CD1B8C300
:10005000D7CFBB9A8DB18F718DB98DB18A618DB9B2
:10006000BA9AB99AB8986A9A08958FB980E48EB905
:10007000769902C0689AFCCF8FB10895CF93C82FAC
:10008000C29AC398892FF1DF8C2FEFDFC39AC29AEF
:10009000CF91089580937A0020917B0030917C006D
:1000A000813049F030F0823049F0833069F42D71AD
:1000B00007C0206C05C02F71226002C02D7328621A
:1000C00030937C0020937B0080917B0090917C009A
:1000D000D5CF8093780020917B0030917C008823DD
:1000E00021F0813039F4386001C0377F30937C00D3
:1000F00020937B0080917B0090917C00BFCFCF93B9
:10010000DF93282FCB01BA01213019F0C0E0D0ECE9
:1001100002C0C0E0D0EEE22FF0E0EE0FFF1FEE0FC6
:10012000FF1FE459FF4F608371838283938320E034
:1001300030E040E054E429D220E030E044E352E4EF
:1001400002D169D1CE01862B972BDF91CF9196CF2B
:100150008093790020917B0030917C00882321F0EE
:10016000813039F4346001C03B7F30937C002093B0
:100170007B0080917B0090917C0080CF8F929F923A
:10018000AF92BF92CF92DF92EF92FF92CF93DF9325
:10019000C82F4A015B0127E73CEC4BE251E4C50163
:1001A000B401F3D120E030E040E850E4EED133D1A7
:1001B0006B017C01EC2FF0E0EE0FFF1FEE0FFF1F35
:1001C000EC59FF4F80829182A282B382C13019F034
:1001D000C0E0D0E402C0C0E0D0E880917B00909104
:1001E0007C0090624BDFD701C60122E0B695A7954F
:1001F000979587952A95D1F79F738C2B9D2B3EDF82
:10020000C7019F738C2B9D2BDF91CF91FF90EF90B7
:10021000DF90CF90BF90AF909F908F902FCF80E4D2
:1002200091E02CDFE4E6F0E08789908D8064908F88
:10023000878B60E070E080E090E0A0DF60E070E03D
:1002400081E090E09BDF60E070E080E090E057DFCD
:1002500060E070E081E090E052DF80E090E039DF24
:1002600080E090E075CFF5DE29E03EE145EE4A956D
:10027000F1F73A95E1F72A95D1F70000D0DF22E0B7
:1002800038E34EEA4A95F1F73A95E1F72A95D1F726
:1002900083E000DF40E050E26BEC76E480E06EDF6C
:1002A00082ED94E02BD208E010E0C0E9D5E622D23E
:1002B000B80122D0C81BD90B2797BE0180E090E07F
:1002C000D6D0AB01BC0180E059DFC03C8DE5D8073A
:1002D00070F710D2B80110D00796C80FD91FBE0111
:1002E00080E090E0C4D0AB01BC0180E047DFC139C1
:1002F00085E6D80770F3D9CF97FB072E16F4009444
:1003000006D077FD08D00BD007FC05D03EF49095C1
:1003100081959F4F0895709561957F4F0895AA1B11
:10032000BB1B51E107C0AA1FBB1FA617B70710F0E0
:10033000A61BB70B881F991F5A95A9F78095909512
:10034000BC01CD0108950CD0E6C0DED040F0D5D080
:1003500030F021F45F3F19F0C7C0511110C1CAC07D
:10036000EBD098F39923C9F35523B1F3951B550BA3
:10037000BB27AA2762177307840738F09F5F5F4F78
:10038000220F331F441FAA1FA9F333D00E2E3AF0B9
:10039000E0E830D091505040E695001CCAF729D0D3
:1003A000FE2F27D0660F771F881FBB1F2617370722
:1003B0004807AB07B0E809F0BB0B802DBF01FF2752
:1003C00093585F4F2AF09E3F510568F08DC0D7C00B
:1003D0005F3FECF3983EDCF3869577956795B7958C
:1003E000F7959F5FC9F7880F911D9695879597F9A7
:1003F0000895E1E0660F771F881FBB1F6217730720
:100400008407BA0720F0621B730B840BBA0BEE1F34
:1004100088F7E095089598D088F09F5790F0B92F0D
:100420009927B751A0F0D1F0660F771F881F991F49
:100430001AF0BA95C9F712C0B13081F09FD0B1E07F
:1004400008959CC0672F782F8827B85F39F0B93F8F
:10045000CCF3869577956795B395D9F73EF490954B
:100460008095709561957F4F8F4F9F4F0895E894C9
:1004700009C097FB3EF490958095709561957F4FEC
:100480008F4F9F4F9923A9F0F92F96E9BB2793959A
:10049000F695879577956795B795F111F8CFFAF4AA
:1004A000BB0F11F460FF1BC06F5F7F4F8F4F9F4FDB
:1004B00016C0882311F096E911C0772321F09EE839
:1004C000872F762F05C0662371F096E8862F70E09F
:1004D00060E02AF09A95660F771F881FDAF7880F79
:1004E0009695879597F9089597F99F6780E870E04A
:1004F00060E008959FEF80EC089500240A9416169A
:10050000170618060906089500240A941216130601
:10051000140605060895092E0394000C11F488238F
:1005200052F0BB0F40F4BF2B11F460FF04C06F5FAB
:100530007F4F8F4F9F4F089557FD9058440F551F81
:1005400059F05F3F71F04795880F97FB991F61F055
:100550009F3F79F087950895121613061406551FCC
:10056000F2CF4695F1DF08C0161617061806991F38
:10057000F1CF86957105610508940895E894BB272D
:1005800066277727CB0197F908950AD0C4CFB5DF46
:1005900028F0BADF18F0952309F0A6CFABCFEFCF44
:1005A000CBDFA8F39923D9F35523C9F3950F50E076
:1005B000551FAA27EE27FF27BB270024089467951D
:1005C00020F4E20FF31FB41F0A1E220F331F441F33
:1005D000AA1F6695A9F7779530F4F30FB41F0A1E8A
:1005E000121E08F46395330F441FAA1F221F76952D
:1005F00099F7879520F4B40F0A1E121E631F440F4B
:10060000AA1F221F331F8695A9F7862F712D602DF3
:1006100011249F5750408AF0E1F088234AF0EE0FF2
:10062000FF1FBB1F661F771F881F91505040A9F7FF
:100630009E3F510570F058CFA2CF5F3FECF3983E3C
:10064000DCF3869577956795B795F795E7959F5F66
:10065000C1F7FE2B880F911D9695879597F9089500
:100660008F929F92AF92BF92CF92DF92EF92FF92C2
:10067000CF93DF93EC01688179818A819B81611539
:1006800071058105910521F464E279ED8BE597E030
:100690002DE133EF41E050E055D049015A0127EAFE
:1006A00031E440E050E035D06B017C012CEE34EFBA
:1006B0004FEF5FEFC501B4012CD0DC01CB018C0DF5
:1006C0009D1DAE1DBF1DB7FF03C00197A109B04816
:1006D00088839983AA83BB839F77DF91CF91FF9013
:1006E000EF90DF90CF90BF90AF909F908F90089544
:1006F000B7DF089580E690E0B3DF0895A0E0B0E0B2
:100700008093600090936100A0936200B0936300B7
:100710000895EE27FF27AA27BB2708C0A20FB31F03
:10072000E41FF51F220F331F441F551F9695879511
:100730007795679598F37040A9F7009799F7BD01F1
:10074000CF010895052E97FB16F400940FD057FDA6
:1007500005D014D007FC02D046F408C0509540954F
:10076000309521953F4F4F4F5F4F0895909580955D
:10077000709561957F4F8F4F9F4F0895A1E21A2E7C
:10078000AA1BBB1BFD010DC0AA1FBB1FEE1FFF1F35
:10079000A217B307E407F50720F0A21BB30BE40B85
:1007A000F50B661F771F881F991F1A9469F76095CC
:1007B0007095809590959B01AC01BD01CF01089586
:0407C000F894FFCFDB
:0407C4000100000030
:00000001FF
